:100000000C94F1030C9438040C9438040C943804C8
:100010000C9438040C9438040C9438040C94380470
:100020000C9438040C9438040C949A2C0C946E2D77
:100030000C94FD260C9438040C9438040C94380469
:100040000C9438040C9438040C9438040C94380440
:100050000C9438040C9470270C9438040C943804D5
:100060000C9438040C9438040C9438040C94380420
:100070000C9438040C9438040C9438040C94380410
:100080000C9438040C9438040C9438040C94380400
:100090000C9438040C9438040C9438040C943804F0
:1000A0000C9438040C9438040C943804002000108C
:1000B0000022021200230313002404140025051556
:1000C0000026061600270717002808180029091916
:1000D000002A0A1A002B0B1B002C0C1C002D0D1DD6
:1000E000002E0E1E002F0F1F0050304000513141D6
:1000F00000523242005333430054344400553545D6
:100100000056364600573747005838480059394995
:10011000005A3A4A005B3B4B005C3C4C005D3D4D55
:10012000005F3F4F008060700081617100826272E9
:100130000083637300846474008565750086667649
:10014000008767770088687800896979008A6A7A09
:10015000008B6B7B008C6C7C008D6D7D008F6F7FC6
:1001600000B090A000B191A100B292A200B393A3FD
:1001700000B494A400B595A500B696A600B797A7BD
:1001800000B898A800B999A900BA9AAA00BB9BAB7D
:1001900000BD9DAD00BF9FAF0120001001220212E3
:1001A0000123031301240414012505150126061655
:1001B000012707170128081801290919012A0A1A15
:1001C000012B0B1B012D0D1D012E0E1E0150304069
:1001D000015131410152324201563646015A3A4AE2
:1001E000015B3B4B015C3C4C015D3D4D015E3E4E75
:1001F000015F3F4F29000000BE00BD00805F815FAE
:10020000CA5CC95CAC00AE00AB00A800AA00A900A3
:10021000490035001E001F0020002100220023009D
:1002200024002500260027002D002E002A004B0068
:100230002B0014001A000800150017001C001800FD
:100240000C00120013002F00300031004E00390066
:1002500004001600070009000A000B000D000E0044
:100260000F0033003400520028004A00E100000073
:100270001D001B00060019000500110010003600CB
:10028000370038005100E5004C00E000E200E300D8
:100290000000000000002C00000000000000E7004B
:1002A0000151E40050004F00010000003A003B0003
:1002B0003C003D003E003F00400041004200430042
:1002C000440045000100010001000100010001009F
:1002D0000100010001000100010001000100010016
:1002E00001000100C25CC35CC95CC55CC75CCB5C3F
:1002F00001000100010001000100010001000100F6
:1003000001000100C45CCA5CC65CC85CCC5C010036
:1003100001000100010001000100010001000100D5
:1003200001000000010001000100010001000100C6
:1003300001000100010001000100010001000100B5
:1003400001000100000000000000010000000000AA
:10035000000001000100010001000100290000006F
:100360003A003B003C003D003E003F0040004100A1
:100370004200430044004500490035001E001F00B4
:100380002000210022002300240025002600270051
:100390002D002E002A004B002B0014001A0008002C
:1003A000150017001C0018000C00120013002F008D
:1003B000300031004E00390004001600070009002B
:1003C0000A000B000D000E000F0033003400520035
:1003D00028004A00E10000001D001B000600190073
:1003E0000500110010003600370038005100E5000C
:1003F0004C00E000E300E2000000000000002C00E0
:10040000000000000000E6000351E40050004F002F
:1004100001000000BE00BD00825F835FCA5CC95C52
:10042000AC00AE00AB00A800AA00A90001000100CA
:1004300001000100010001000100010001000100B4
:10044000010001000100010001000100C25CC35C69
:10045000C95CC55CC75CCB5C010001000100010008
:10046000010001000100010001000100C45CCA5C40
:10047000C65CC85CCC5C0100010001000100010009
:100480000100010001000100010000000100010065
:100490000100010001000100010001000100010054
:1004A0000100010001000100010001000000000046
:1004B0000000010000000000000001000100010038
:1004C0000100010000000000000000002A2B2800AD
:1004D00000000000000000000000000000000029F3
:1004E000000000002C1E3420212224342627252E33
:1004F000362D3738271E1F2021222324252633336B
:10050000362E37381F0405060708090A0B0C0D0E96
:100510000F101112131415161718191A1B1C1D2F62
:100520003130232D350405060708090A0B0C0D0E82
:100530000F101112131415161718191A1B1C1D2F42
:100540003130354C000000000000000000000000C9
:10055000000000000000000000000000000000009B
:1005600000000000000000007E0F00D4FFFFFFC766
:1005700000000078000101010101010101010202F6
:100580000202020202020203030303030303030441
:10059000040404040404050505050506060606060C
:1005A000070707070708080808090909090A0A0AC6
:1005B0000B0B0B0C0C0C0D0D0D0E0E0E0F0F0F1068
:1005C00010111111121213131414151516161717F2
:1005D000181819191A1A1B1B1C1D1D1E1E1F20205E
:1005E000212222232424252626272829292A2B2CA8
:1005F0002D2D2E2F30313232333435363738393ACB
:100600003B3C3D3E3F404142434445464748494AC2
:100610004C4D4E4F50515354555658595A5B5D5E90
:100620005F616264656668696B6C6D6F707273752B
:1006300077787A7B7D7E8082838587888A8C8E8F8F
:1006400091939596989A9C9EA0A2A3A5A7A9ABADBD
:10065000AFB1B3B5B7BABCBEC0C2C4C6C9CBCDCFAB
:10066000D1D4D6D8DBDDDFE2E4E7E9EBEEF0F3F559
:10067000F8FAFDFF18034B0065007900630068007D
:1006800072006F006E002000510031000000120364
:100690004B00650079006300680072006F006E0017
:1006A00000000403090409025B00030100A0FA0929
:1006B0000400000103010100092111010001224091
:1006C000000705810308000109040100020300007E
:1006D00000092111010001222200070582032000E8
:1006E00001070503032000010904020001030000C3
:1006F00000092111010001226D000705840320007B
:100700000112010002000000083434000100010160
:100710000200010660FF0961A1010962150026FFC0
:10072000009520750881020963150026FF009520B9
:1007300075089102C005010980A101850319012AEC
:10074000B700150126B700950175108100C0050C92
:100750000901A101850419012AA002150126A002A0
:10076000950175108100C005010906A101850605E6
:100770000719E029E7150025019508750181020593
:1007800007190029EF1500250195F0750181020573
:1007900008190129059505750191029501750391C7
:1007A00001C005010906A101050719E029E71500A7
:1007B00025019508750181029501750881010507DC
:1007C000190029FF150026FF009506750881000510
:1007D0000819012905950575019102950175039187
:1007E00001C011241FBECFEFDAE0DEBFCDBF04B6DB
:1007F00003FE27C08091E7059091E805A091E905E7
:10080000B091EA058730904BA740B04BD1F41092DD
:10081000E7051092E8051092E9051092EA0514BE6A
:1008200084B7877F84BF0FB6F894A8958091600045
:10083000886180936000109260000FBEE0E0F8E3F2
:10084000099513E0A0E0B1E0EEE8F1E602C0059002
:100850000D92A031B107D9F725E0A0E1B3E001C0C6
:100860001D92A73EB207E1F70E94CC140C947C3095
:100870000C9400001F93CF93DF93182FD62F0E9464
:10088000EC21C82F882339F0111105C081E0D11166
:1008900084E00E94020A8C2FDF91CF911F9108956E
:1008A000CF93FB0181382FE5920719F138F4803896
:1008B0009F4599F0C1E08C2FCF91089582382FE5A4
:1008C0009207E9F083389F45A9F7C28183EECC23D4
:1008D00031F10E94BD0688E019C08281882331F081
:1008E0008FE992E00E94CA25C0E0E5CF90E080E069
:1008F000F9CF82818823D1F380EA92E0F3CFC281DD
:1009000083EECC2331F00E94BD068BE20E94BD062F
:10091000EBCF0E9403078BE20E940307CCCF0E941B
:10092000030788E0F9CF81E008950C9450040895FE
:100930000C9497041F93CF93DF9300D000D00F92B5
:10094000CDB7DEB749835A836B8330911203898117
:100950009A8131111DC06623B9F02223A9F00E94AB
:10096000AE0A182F682F89819A810E945A0A6981DC
:100970007A81812F0F900F900F900F900F90DF9141
:10098000CF911F910C94FB220E94860A182FEFCF63
:100990000E94AE0A69817A81EDCFFC01262F408149
:1009A00051816281738184810C949A0481E008955D
:1009B000CF93DF93EC0160E00E94CD04BE01DF9194
:1009C000CF910C949804E1E0F0E0DF0102C0AA0F9F
:1009D000BB1F6A95E2F7BD01DF0102C0AA0FBB1F72
:1009E0004A95E2F76A2B01C0EE0F2A95EAF7962F97
:1009F0009823961302C08E2B0895E0958E230895B8
:100A0000242F462F682F809137030E94E3040C9413
:100A1000170A0E941A130E9471060E94231B0C944D
:100A2000351380E00E94F7210C9438130E94C31AFA
:100A300080E00E94720681E00C94411B08950895A5
:100A40000E94AF090E941F052FEF84E39CE0215014
:100A500080409040E1F700C000000C9494270F9371
:100A60001F93CF93DF938C0161E00E94CD04EC01D2
:100A7000B8010E946F1F882309F441C0B801CE015C
:100A80000E9495048823D9F1B801CE010E945C240C
:100A90008823A9F1B801CE010E94C220882379F1F0
:100AA000B801CE010E94C623882349F1B801CE01C6
:100AB0000E947E1E882319F1F8018281882361F04B
:100AC000CA35FDE5DF0721F170F4C115ECE5DE075D
:100AD000A1F0CE3DDC45C9F0C801DF91CF911F9157
:100AE0000F910C949304CB358DE5D807A1F0CC354C
:100AF000DD4591F70E94460FEFCF0E94200580E070
:100B0000DF91CF911F910F9108950E94FF0FF7CFB2
:100B10000E944F0FE1CF0E94520FDECF0C941E05B2
:100B20000E948E250E94720680E00E94411B0C9458
:100B30008E05DF92EF92FF920F931F93CF93DF9377
:100B4000E82FF0E0EC53FB4FD490282F2695269504
:100B5000269530E0F901EC59FA4F0491877010E0C6
:100B6000082E02C0159507950A94E2F70170112727
:100B7000F901EC5AFA4FE490F12C082E02C0F594DA
:100B8000E7940A94E2F791E0E922FF24F901EC5B93
:100B9000FA4FC491D0E002C0D595C7958A95E2F787
:100BA000C170DD270115110519F081EE0E94BD0607
:100BB000E114F10419F086EE0E94BD068D2D0E940D
:100BC0004207EF2819F086EE0E940307012B19F067
:100BD00081EE0E940307CD2B51F08CE2DF91CF9183
:100BE0001F910F91FF90EF90DF900C944207DF91DF
:100BF000CF911F910F91FF90EF90DF900895EF92AA
:100C0000FF920F931F93CF93DF93EC01162F0AE00F
:100C10008881882309F454C0813009F04EC089814D
:100C2000813099F47E0122E0E20EF11C8A810E945B
:100C30004207E7012196812F815050F3EFE9FFE051
:100C40003197F1F700C00000F7CF823041F47E0108
:100C500082E0E80EF11C8A810E94BD06EACF833053
:100C600041F47E01E2E0EE0EF11C8A810E9403074E
:100C7000E0CF843011F02196DDCF2A81229690E0DA
:100C800080E0AE014F5F5F4F2053330B2A303105B8
:100C900048F0019778F2EFE9FFE03197F1F700C0F3
:100CA0000000F7CF089FB001099F700D1124C90102
:100CB000860F971F2981EA01E4CF0E949905BACFD8
:100CC000DF91CF911F910F91FF90EF90089560E019
:100CD0000C94FF0508950C946A0681E008950C9425
:100CE0006D060895CF93C82F0E946B068C2FCF916D
:100CF0000C946F06CF93DF93CDB7DEB72B970FB66B
:100D0000F894DEBF0FBECDBF4F83588769877A87BF
:100D10008B8761110E94940E1E821D8285E0FE0168
:100D20003796DE01119601900D928A95E1F78C813C
:100D30009D81892B89F449815A816B817C818D81C8
:100D40009E810E94B50D2B960FB6F894DEBF0FBEA4
:100D5000CDBFDF91CF91089589819A8189238F3FFB
:100D600051F3CE0101960E94D6048111E4CFEBCF5E
:100D7000FC01808191810C94DB0ACF93C82F8823DA
:100D800009F43FC08CEF8C0F813AA0F46C2F809156
:100D90005602909157020E94F425882329F08C2F47
:100DA0000E94560E0E94C40E8C2F0E944F0ECF91AF
:100DB0000C94C40E80E28C0F883048F4C77081E038
:100DC00001C0880FCA95EAF70E94770EF0CFEBE5D5
:100DD000EC0FE33040F4F0E0E855FD4F808190E007
:100DE000CF910C94B425C85AC73158F4EC2FF0E0D9
:100DF000EE0FFF1FE658FD4F80819181CF910C943B
:100E0000CA25CF910895882329F19CEF980F913A34
:100E100020F40E94560E0C94C40E90E2980F983065
:100E200050F4877091E001C0990F8A95EAF7892FF5
:100E30000E947D0EF0CF9BE5980F933020F490E058
:100E400080E00C94B425885A873120F490E080E04B
:100E50000C94CA2508951F93CF93DF93182FEB01AD
:100E60000E94BD06209731F4812FDF91CF911F9111
:100E70000C9403078FE99FE00197F1F700C0000091
:100E80002197F0CF70E060E0893311F460E570E005
:100E90000C942B07882321F00E94770E0C94C40E2B
:100EA0000895882321F00E947D0E0C94C40E0895AD
:100EB000BF92CF92DF92EF92FF920F931F93CF9347
:100EC000DF936C01D62FC72FFC011281F580F294BD
:100ED0009FE0F9220E946D0EE82E8823B9F0E12EE2
:100EE0001123A1F08C2F807F803421F080E28D0FC0
:100EF0008830B0F080911F0482FD12C082E00E9411
:100F0000150F0E946D0E91E0E82EE926BC2EB294DA
:100F10008FE0B822EB2DF0E0E258FF4C0C946A2FE2
:100F2000E12CF4CF0C2F0F70C07F11F00295007FE1
:100F3000112399F0002359F080E28D0F883010F0D2
:100F4000D11107C0802F0E94770E0E94C40E8D2FF2
:100F500041C0802F0E94870EF8CF8D2F0E9403077B
:100F6000002309F43FC080E28D0F883010F0D111CA
:100F700004C0802F0E947D0E03C0802F0E948D0E22
:100F80000E94C40E2FC00C2F0F70C07FC03211F012
:100F90000295007FDD2381F0D13009F469C011236F
:100FA00009F473C0FF2009F469C0F601858180FF50
:100FB000CECF8F70858362C080911F0482FF38C0BE
:100FC000112359F0002329F0802F0E94770E0E94F0
:100FD000C40E80E00E94BD0605C080E00E940307A9
:100FE0000111C7CFEB2DE850FF0B349720F40E947E
:100FF0008E250E947206EE2009F452C10E94690EED
:1010000080FD4EC1F60112820E94630E0E94280AE2
:10101000C6010E9471090E94630EDF91CF911F915A
:101020000F91FF90EF90DF90CF90BF900C94330A18
:10103000112389F0F11006C00E94A70E802B0E9498
:101040004A07D0CFF1E0FF12F7CF0E94A70E802B06
:101050000E94AD0EC7CFF11006C00E94BA0E802FBD
:101060000E945107BFCF21E0F21609F4BBCFF5CFA4
:10107000112331F035E03F1508F4B4CF802FDFCFD6
:1010800084E08F1508F4AECFEACFFF2041F3D933C7
:1010900049F4FFEF27EE33E0F15020403040E1F714
:1010A00000C000008D2F0E9403079CCF8C2F8695D7
:1010B0008695837069F0813009F094CF8D2F9C2F35
:1010C0009370111102C090E080E00E94CA258ACF7F
:1010D0008D2F9C2F9370111102C090E080E00E9430
:1010E000B42580CF8C2F837079F511117BCF4D2FD4
:1010F000429546954770440F440F8D2F8F70042EF4
:1011000001C0880F0A94EAF72D2F2071D4FF07C081
:101110002FE030E001C0220F4A95EAF72095C695EE
:10112000C695C370822BC23049F058F4C13019F013
:101130000E94090A57CF0E94040A54CF0E940E0A47
:1011400051CF0E94020A4ECF8695112311F08C2FA9
:101150008170882309F446CF4D2F429546954770FC
:10116000440F440F8D2F8F70042E01C0880F0A94F6
:10117000EAF72D2F2071D4FF07C02FE030E001C027
:10118000220F4A95EAF72095C695C695C370822B23
:10119000C23049F058F4C13019F00E944F0A22CFF2
:1011A0000E944A0A1FCF0E94540A1CCF0E94170AAD
:1011B00019CFCF70112329F08C2F0E94280A8D2F70
:1011C0003ECF8D2F0E9451078C2F0E94330A0ACFE9
:1011D000D23F51F160F4D03FB9F0D13F81F01123FB
:1011E00009F449C0F110B3CE8C2F8F7121C0D33FC9
:1011F00011F1D43FA1F780911F0482FF26C08C2FEC
:101200008F71112311F314C0112349F084E08F155D
:1012100008F4E8CE8C2F8F710E943F0AE3CE95E050
:101220009F1508F4DFCEF6CF8C2F8F711111CDCF23
:101230000E94280AD7CE112329F08C2F8F710E948B
:10124000200AD0CE0E941D0ACDCE112349F0CF71C5
:101250008C2F0E94280A63E08C2F0E94FA0EC2CEC7
:1012600081E00E94150FE1E0EF1508F0BBCE82E0AF
:101270000E94150FB7CEF1100ACF8C2F8F71A5CF1A
:101280004C2F4F706D2FC6010E940C110E94090B4C
:10129000A9CE4C2F4F706D2FC6010E940F11A2CE08
:1012A000DF91CF911F910F91FF90EF90DF90CF9042
:1012B000BF9008950F931F93CF93DF93EC01688144
:1012C00079818A810E94E50A8C010E94590A0E9454
:1012D000010AB801CE01DF91CF911F910F910C94BB
:1012E0005807CF93DF93EC018B819C81892B29F0E8
:1012F0008881998189238F3F59F4DF91CF91089597
:10130000CE010E945A09CE01DF91CF910C94D804EE
:10131000CE010E942F058111F3CF0E946D0E88230C
:1013200061F38A81882349F380911F0482FDE5CF10
:1013300082E0DF91CF910C94150F90E080E00E9445
:10134000B42590E080E00E94CA250E94940E0E947D
:10135000A40E0C94C40E0E945D0E0C949D090E9474
:10136000840E0C94AB09E92FE295EF70E250EE3059
:1013700070F4F0E0E257FF4C0C946A2F803F19F0B4
:1013800020F4883E20F481E00895843FE1F380E07A
:101390000895883EC0F3813FD1F7F5CF93FB8827AE
:1013A00080F90895FC01808191810E94DB0A0C94F0
:1013B000B309CF93DF9300D000D00F92CDB7DEB743
:1013C0000F900F900F900F900F90DF91CF91089595
:1013D000CF93DF9300D000D000D0CDB7DEB72696F4
:1013E0000FB6F894DEBF0FBECDBFDF91CF91089549
:1013F00008950C94F8090E94F909809338030C941D
:101400009D0908950C94FB0990913803892B0C9445
:10141000FB099091380389230C94FB0990913803C0
:1014200089270C94FB090C94F8090C94130A0E9468
:10143000150A809337030C949D0980E00C94170AD9
:1014400091E001C0990F8A95EAF7892F0C94170A49
:1014500021E030E001C0220F8A95EAF7809137033E
:10146000822B0C94170A21E030E001C0220F8A95EC
:10147000EAF720958091370382230C94170A21E024
:1014800030E001C0220F8A95EAF780913703822766
:101490000C94170A90913703892B0C94170A90919A
:1014A000370389230C94170A9091370389270C94EA
:1014B000170A08952FE0929F800D1124982F97709E
:1014C00041E001C0440F9A95EAF786958695869586
:1014D00093E0899FF0011124ED5EFC4F90E080E0E5
:1014E00070E05191DF0111979B01082E02C03695E3
:1014F00027950A94E2F72170219525272423252793
:101500002C9301968330910561F708952FE0929F07
:10151000800D1124982F977086958695869523E0E7
:10152000829FF0011124ED5EFC4F50E040E080E02E
:10153000219130E0092E02C0369527950A94E2F7F2
:1015400021703327042E01C0220F0A94EAF7822B60
:101550004F5F5F4F4330510559F70895CF92DF92A7
:10156000FF920F931F93CF93DF936C01009137038A
:1015700080913803082BC7E0D0E010E0FC2EC801B2
:101580000C2E02C0959587950A94E2F780FD0CC059
:101590002197A0F7F12C8F2DDF91CF911F910F9103
:1015A000FF90DF90CF900895B6018C2F0E942212F9
:1015B000019771F3F0CFCF93DF93EC010E94AE0A55
:1015C000BE01DF91CF910C9422121F93CF93DF9332
:1015D000EB0190911203992331F0CB01DF91CF9170
:1015E0001F910C94DB0A882379F0CB010E94AE0A8C
:1015F000182F682FCE010E945A0ABE01812FDF9159
:10160000CF911F910C942212CB010E94860A182FB1
:10161000F4CFEF92FF920F931F93CF93DF938C0140
:10162000892B81F0F12CEE24E394E8012196F80156
:101630008491843770F4843008F05FC08130B1F059
:101640008230A1F1DF91CF911F910F91FF90EF9028
:101650000895853709F44CC008F43DC09CE7980F05
:10166000903780F78F770E94030749C00E5F1F4FA6
:10167000FE01849190E2980F983060F48770FE2DFF
:1016800001C0FF0F8A95EAF78F2F0E94970E0E94E4
:10169000C40E02C00E94BD068F2D815030F2EFE9CA
:1016A000FFE03197F1F700C00000F7CF0E5F1F4F4A
:1016B000FE01849190E2980F983050F48770FE2DCF
:1016C00001C0FF0F8A95EAF78F2F0E949D0EDFCF92
:1016D0000E940307E1CF0E5F1F4FFE01C491C1506E
:1016E000D8F28FE99FE00197F1F700C00000F7CF33
:1016F0000E5F1F4FFE01F490CFCF0E94BD068E01FA
:10170000CBCF1F93CF93DF93C091390316E0809125
:101710003A038C1304C0DF91CF911F910895D0E05C
:101720001C9FF0011D9FF00D1124E55CFC4F4081D2
:10173000518162817381848195810E94E80921969B
:10174000C770E5CF40916B0350916C0360916D03BE
:1017500070916E0380916F03909170030C94E8096F
:10176000FF920F931F93CF93DF9380917003807F3D
:10177000D1F480916D038823B1F0809139031091E9
:101780003A0360916B0370916C03A0916E03B0916A
:101790006F03062F0723C0915402D091550296E0A3
:1017A000F92E181306C0DF91CF911F910F91FF9072
:1017B000089590E0109711F00F3F19F4019687708B
:1017C000F0CFF89E9001F99E300D1124F901E55CEF
:1017D000FC4F41814713F2CF40814613EFCF428146
:1017E0004111ECCF438154814A1B5B0B4C175D07C1
:1017F00028F7809170038F70806180937003F901E6
:10180000E05CFC4F80818F70806180838BE693E089
:101810000E947109DF91CF911F910F91FF900C945D
:10182000810BAF92BF92CF92DF92EF92FF920F9314
:101830001F93CF93DF93CDB7DEB761970FB6F894C0
:10184000DEBF0FBECDBF8C0185E0F801DE011D9625
:1018500001900D928A95E1F7F801E2808BE6C82E9F
:1018600083E0D82E60916E0370916F03611571054E
:1018700009F45FC190916B0320916C03892F82233F
:101880008F3F09F456C140815181A380B480F0900C
:101890006D03F501E61BF70BBF01E0915402F091D7
:1018A0005502FF2009F4F6C080917003382F307F75
:1018B0006E177F0708F0AFC0311179C0FE2C2513D9
:1018C00023C0941321C0E1101FC08F7080618093EA
:1018D00070030E94A20BC6010E94710980917003DF
:1018E000F80185838F2D61960FB6F894DEBF0FBE89
:1018F000CDBFDF91CF911F910F91FF90EF90DF90BF
:10190000CF90BF90AF900895AB2829F0842F852306
:101910008F3F09F027C180E0F82FF170DF2E80FFA4
:101920003CC08091390320913A0336E0821315C000
:101930004D875E878D859E850E94DB0A292F229523
:101940002F702230F0F0243018F59F70F1F0F8017C
:101950009581907FD1F4D12C1EC090E0389FF0018A
:10196000399FF00D1124E55CFC4F6181651306C0C1
:101970006081641303C062816E110FC0019687708D
:10198000D5CF9F7011F0882331F3805E883018F333
:10199000C8010E947109FD2CA5CFEE2009F4A2CF49
:1019A00080917003816080937003F12C9BCF25138D
:1019B00006C0941304C0F801EE2009F487C0C801E2
:1019C0000E94D209882319F1EE2009F18091700359
:1019D000803270F020916B0330916C0338872F8335
:1019E0001986BB86AA868C87CE0107960E9471094C
:1019F00086E0F801ABE6B3E001900D928A95E1F73D
:101A00000E94B00B0E94A20BFF24F3946BCFC8017D
:101A10000E947109F9CF311113C07A2DB98AA88AB1
:101A20006E2D89890E94D9098BE693E00E94710985
:101A300086E0F60111928A95E9F70E94A20BB5CFD4
:101A400025130FC094130DC0E1100BC0F80185835E
:101A5000C8010E94710986E0F60111928A95E9F7A2
:101A600041CFC8010E94D209882389F2EE2079F281
:101A700080917003803208F4BBCF20916B033091CA
:101A80006C033A8329831B82BD82AC828E83CE0194
:101A90000196ACCF6E177F0708F03EC0FE2CEE20FB
:101AA00009F4B5CF25132AC0941328C08091700380
:101AB00080FD1BC0982F907FC1F0F8018583903F77
:101AC00031F0982F907F905F8F70892B8583C801AC
:101AD0000E94710986E0F801ABE6B3E001900D9237
:101AE0008A95E1F70E94A20BFDCE86E0F801ABE6F5
:101AF000B3E001900D928A95E1F7F4CEC8010E94FF
:101B0000D209811175CF8091700381608093700339
:101B1000C8010E947109E6CE7A2DB98AA88A6E2D75
:101B200089890E94D90986E0F60111928A95E9F720
:101B3000D9CFEE2009F46BCFC8010E94D209F82E4C
:101B4000882309F464CF86E0F801ABE6B3E00190A6
:101B50000D928A95E1F78BE693E00E94B8060E9409
:101B6000B00BC0CF81E08E25D7CE1F93CF93DF93EC
:101B7000CDB7DEB72C970FB6F894DEBF0FBECDBF42
:101B80004F83588769877A878B879C87CE01079612
:101B90000E94110C882369F08A859B85892B39F076
:101BA0004F815885842F85238F3F09F071C016E03F
:101BB0005FC086E0FE013796DE01119601900D921E
:101BC0008A95E1F78A859B85892B89F38F81988592
:101BD00089238F3F61F320913A0330E0C9010196D8
:101BE00087709927409139034817190671F40E94AC
:101BF000AF0910923A031092390386E0EBE6F3E066
:101C0000DF011D928A95E9F7D2CF96E0929FD0012D
:101C1000939FB00D1124A55CBC4FFE01319601903D
:101C20000D929A95E1F780933A030E94810BBFCF02
:101C3000819FC0011124855C9C4F0E94110C882358
:101C4000E9F0E09139031E9FF0011124E55CFC4F9F
:101C50004081518162817381848195810E94E8096C
:101C60008091390390E0019687709927809339031A
:101C70008091390390913A038913DACF2C960FB6ED
:101C8000F894DEBF0FBECDBFDF91CF911F910895B5
:101C900069857A858B859C850E94E80988CF682FA5
:101CA00080915602909157020C947426682F80916F
:101CB0005602909157020C947F2680915602909183
:101CC00057020C948A268091710385958595859598
:101CD00008958091710387700895909171039770B2
:101CE00081E009F480E00895809195030895909132
:101CF0009503892B80939503089580959091950382
:101D000098239093950308951092950308959091C8
:101D10009403892B80939403089580959091940364
:101D200098239093940308951092940308959091AA
:101D30009303892B80939303089580959091930347
:101D4000982390939303089510929303089580919C
:101D50007203089508950C94AA0E90911F0492FDA9
:101D600008C090917203981721F0809372030C942D
:101D7000AB0E089580917203882329F010927203AC
:101D800080E00C94AB0E0895E0915602F09157025A
:101D9000809195038083E0915602F09157028081F3
:101DA00090919403892B8083E0915602F091570221
:101DB000808190919303892B808390917203992362
:101DC00081F0E0915602F09157028081892B808347
:101DD00080915602909157020E94E02581110E9445
:101DE000BA0E80915602909157020C949A2508954C
:101DF0000C94F70E90911F0492FD10C098E0899FFB
:101E000090011124622B609371030E94280A809133
:101E100071038595859585950C94F80E0C94280A88
:101E20001092710380E00C94F80E909171038095EC
:101E3000892380937103282F277091F4282F082E6F
:101E4000000C330B9217130659F090911F0492FD6A
:101E500007C08595859585950E94330A0C94100FCF
:101E6000089590911F0492FB222720F9281769F00A
:101E700080FB92F990931F0480911E0490911F049F
:101E80000E947C0F82E00C94150F089580911F042E
:101E900082FB882780F991E089270C94310F81E03B
:101EA0000C94310F80E00C94310F6FEF7FEF90E0D6
:101EB00080E00C94353090E080E00E940130893E53
:101EC0009E4F11F40C94181F80E0089582E090E07A
:101ED0000C94F92F83E090E00C94F92FCF9384E0D9
:101EE00090E00E94F92FC82F82E290E00E94F92F23
:101EF000982F8C2FCF910895CF93C92F682F84E00E
:101F000090E00E9417306C2F82E290E0CF910C9409
:101F10001730AB01BC018FE090E00C942930AB018D
:101F2000BC0183E190E00C94293060E070E0CB01CB
:101F30000C948F0F60E070E0CB010E94890F0C942D
:101F4000950F69EE7EEF90E080E00E94353060E012
:101F500082E090E00E94173060E083E090E00E9411
:101F600017301092380360E084E090E00E94173050
:101F700060E082E290E00E94173060E085E090E04F
:101F80000E94173060E086E090E00E9417306FEF0B
:101F900087E090E00E94173040E050E0BA0188E00E
:101FA00090E00E94293060E08DE090E00E941730C0
:101FB00040E050E0BA0188E190E00E94293060E002
:101FC00087E190E00E94173040E050E0BA018CE1D8
:101FD00090E00E94293070E060E080E290E00E9492
:101FE000353040E050E0BA0188E190E00E942930AD
:101FF00080E00E94311F0E94571F0C949A0F0C948E
:10200000A10F682F8EE090E00C9417300E943927C2
:102010006093A7037093A8038093A9039093AA03E6
:102020006093A3037093A4038093A5039093A603E6
:10203000089585B7806885BF85B7806885BF089596
:10204000089508950C94201008950C9424100E9473
:10205000191080E093E10E9484250E9421100C94C5
:10206000221081E008950C943110089508950E9483
:1020700035100C9436100E9424270E94661F0E947F
:102080001C14EEE1F4E080818068808380911E045E
:1020900090911F040E947C0F0E94F2210C94251045
:1020A0006F927F928F929F92AF92BF92CF92DF9268
:1020B000EF92FF920F931F93CF93DF93CDB7DEB7CD
:1020C0002A970FB6F894DEBF0FBECDBF0E94311421
:1020D00081110E94061027E9E22E23E0F22E10E083
:1020E000712C812F0E943A134C01F701A080B1801E
:1020F000A816B90609F440C08091AB0381FD0E9487
:102100004A13A824B92400E0CC24C394D12CC501DF
:102110008C219D21892B59F10E94331066246394F0
:1021200094012C213D21232B09F4612C882379F083
:102130000E831F8368860E942D278160782F9A87DF
:1021400089874E815F8168858A850E947A06F701BA
:10215000808191818C259D2591838083462D602FE0
:10216000812F0E94171A7394FBE0F715F0F00F5FB0
:10217000CC0CDD1C0F3059F61F5F82E0E80EF11C1D
:10218000163009F0AECF711010C08FEF89838A83AB
:102190001B820E942D278160782F9D838C8349812B
:1021A0005A816B818D810E947A060E94C31A0E9417
:1021B0008E25909196038917D1F00E948E258093E9
:1021C00096032A960FB6F894DEBF0FBECDBFDF91FF
:1021D000CF911F910F91FF90EF90DF90CF90BF9024
:1021E000AF909F908F907F906F900C9472062A967C
:1021F0000FB6F894DEBF0FBECDBFDF91CF911F9118
:102200000F91FF90EF90DF90CF90BF90AF909F9095
:102210008F907F906F90089590E080E008950895EA
:10222000FC01EE0FFF1FEC58FA4F85919491089531
:10223000CF93DF930E942612EC01811520E59207CF
:1022400008F041C0811530E4930708F0B4C0803E27
:10225000910518F5803C910508F09DC0883A9105DC
:1022600070F4853A910508F08EC081309105F9F03F
:102270000097E9F00497D8F4D0E0C0E018C08F3B95
:102280009105D0F7C85AD0E0CC0FDD1FC555DD4F02
:102290000990D881C02DD4640AC08115904258F4A9
:1022A000C11581E0D80718F4C83ED10528F7CE0142
:1022B000DF91CF910895C11590E3D90708F071C05F
:1022C000CE019F706AC0811525E5920758F58115EA
:1022D00034E5930708F09EC0811542E5940750F459
:1022E000C11581E5D80708F469C0DC2FCC27C16F80
:1022F000D06ADDCF982F969596959E01237033274F
:10230000C115D34508F077C0C1E0D0E002C0CC0FC2
:10231000DD1F2A95E2F720E2929FC0011124C82B0D
:10232000D92B67C0C11589E5D807A8F4C11598E570
:10233000D90708F074C0C11526E5D20708F09CCF74
:102340008C2F0E94BD12C82FD0E0DC2FCC27CC27C9
:10235000DF71D062ACCFC1153AE5D30708F464C091
:10236000CE0190568115904208F086CF8D2F8F7147
:102370000E94BD1290E0982F882788279F719C01AA
:102380002C2BE901E6CFC55AD0E0C752DD4FC881FA
:10239000D0E0D0648CCF805C91090E941011EC01D8
:1023A00086CFCE019927D3FF03C0EC01D86C7FCF35
:1023B000EC01D06C7CCFDF70D06A79CFCE01E4E045
:1023C00096958795EA95E1F783702C2F26952695AB
:1023D000237090E2299F90011124382B8C2F837059
:1023E000C1E0D0E002C0CC0FDD1F8A95E2F7C22B1E
:1023F000D32BDC685CCFC1E0D0E002C0CC0FDD1F86
:102400002A95E2F730E2939FC0011124C82BD92B03
:10241000DA684DCFD82FCC27C46FD06A48CFDC2FD5
:10242000CC27C06FD06A43CF8C2F8F700E94BD1213
:1024300034E0D695C7953A95E1F7CF709C2FEC0123
:10244000D06935CF0E94FB220C9418118238910577
:10245000B1F1B0F48133910509F475C048F48932C3
:10246000910509F469C08A32910509F473C0089591
:102470008533910509F459C08933910501F1089517
:10248000833E9105A9F138F4803E9105F9F0823E32
:10249000910549F10895863E9105A9F1873E910580
:1024A000C9F1843E910519F520911F0421FF1FC039
:1024B00080911E0484FD14C087EE90E00895209161
:1024C0001E042370A1F080EE90E0089520911E0478
:1024D00020FD47C030911F0430FF09C024FF44C0D5
:1024E00090E080E004C020911E0422FDF7CF089503
:1024F00020911E0422FD3BC030911F0430FDE3CF2C
:1025000024FFF5CFEDCF20911E0423FFF0CF24FD53
:10251000E7CFD2CF20911E0423FD2CC030911F04A1
:1025200031FFEECF84EE90E0089520911E0425FF48
:10253000DECF89E290E0089520911E0425FFD7CFD9
:1025400085E390E0089520911E0426FFD0CF8AE213
:1025500090E0089520911E0426FFC9CF81E390E00A
:10256000089589E390E0089583EE90E0089582EE67
:1025700090E0089586EE90E0089590911E0492FFF9
:1025800006C0282F28712830F9F4877F846093FFD4
:1025900006C0282F28712831F1F4877E84612091AC
:1025A0001F0420FF06C0382F38713830D9F4877FD8
:1025B000816021FF06C0282F28712831D1F4877E41
:1025C000816194FD877E0895282F24712430F9F6C7
:1025D0008B7F8860DCCF282F2471243101F78B7E1C
:1025E0008861DDCF382F3171313019F78E7F8860E7
:1025F000E0CF282F2171213121F78E7E8861E1CF34
:1026000080E008950C94550F0E9431148FE39CE9EB
:102610000197F1F700C000000E94311480E00E9491
:102620003A1380FF04C00E9402130C94942708956B
:102630000C9404130E945B0F811102C00E94FF0FD3
:102640000E94660F8093AB030E946E0F90931F044D
:1026500080931E040E9418130E946A0F0E94020AAF
:10266000809137030C94150A08950C94341308953F
:102670000C94371390E0880F991FDC01A45DBB4FC9
:10268000FC01E259FD4F2D913C9180819181822383
:1026900093230895089580EA8A95F1F7089500C07C
:1026A00008950C944B1390E0880F991F442399F0E0
:1026B000805E9B4FFC018081918121E030E002C06F
:1026C000220F331F6A95E2F72823392381E0232B59
:1026D00009F480E00895845D9B4FECCFF894E82FD7
:1026E000E295EF70F0E031A1282F2F7081E090E0AB
:1026F00001C0880F2A95EAF7982F9095932391A30C
:1027000092A1892B82A378940895CF93DF93CCED87
:10271000D2E089918F3F11F00E946E1382E0CB3E90
:10272000D807B9F7CBEED2E089918F3F11F00E9424
:102730006E1382E0C13FD807B9F7DF91CF910895BA
:10274000AF92BF92CF92DF92EF92FF920F931F93BF
:10275000CF93DF93D82EE92EF62E8A01C62FD0E034
:10276000CE0184529D4F5C01EC0128812F3F09F47A
:1027700058C0F894E22FE295EF70F0E031A12F708D
:1027800081E090E001C0880F2A95EAF7932F982BFB
:1027900091A392A18095892382A378940E944F13DC
:1027A000ABEEB2E0ED2DFE2D61EF72E0E12C6801A1
:1027B000C094D0944D91808191814F3F69F1242F35
:1027C00022952F7030E0E90128A130E04F7002C05F
:1027D000359527954A95E2F720FD1EC0802B912B59
:1027E00091838083EE24E39432966A177B0711F776
:1027F000F50180818F3F11F00E946E136E2D8F2D99
:10280000DF91CF911F910F91FF90EF90DF90CF90CC
:10281000BF90AF900C9451138C219D2191838083A4
:10282000E3CFDF91CF911F910F91FF90EF90DF9059
:10283000CF90BF90AF9008950E9485138CE0ECE29A
:10284000F4E0DF01982F1D929A95E9F7E0E2F4E0B9
:10285000DF011D928A95E9F786E00E9486140C94A8
:102860000905CF92DF92FF920F931F93CF93DF93CF
:10287000CDB7DEB72C970FB6F894DEBF0FBECDBF35
:102880008E010F5F1F4F8CE0F80111928A95E9F7D6
:10289000F12CCC24C394D12CA6016F2DC8010E9429
:1028A000A013F394CC0CDD1CFFE0FF12F5CF4CE03D
:1028B00050E0B80180E294E00E94DC2FFF24F39402
:1028C000009709F4F12C892B41F08CE0F801A0E28B
:1028D000B4E001900D928A95E1F72F2D46E06CE26D
:1028E00074E080E294E00E9487140E9411058F2D0D
:1028F0002C960FB6F894DEBF0FBECDBFDF91CF91FF
:102900001F910F91FF90DF90CF9008950895FF924F
:102910000F931F93CF93DF93F82E092F162FD72FE6
:10292000C42F222349F081E08093AE030E942D271B
:102930009093AD038093AC038091AE038823A1F004
:102940008091AC039091AD030E944527059760F0FC
:10295000EF2DF02FA12FBD2F90E080E0D0E08C175D
:102960009D0744F01092AE03DF91CF911F910F911C
:10297000FF900895219131912D933D930196EFCFD2
:102980000E946F290E943B100C947B290E947F2992
:102990000E9450100C9499290E94B6260E94562934
:1029A0000E9427100E94C0140E94C6140E94371073
:1029B000FBCFEF92FF920F931F93CF93DF93EB0127
:1029C000E82FD11110C0442321F0F0E0EC58FA4F69
:1029D000E4916E2F7E2F8E2FDF91CF911F910F915B
:1029E000FF90EF9008950D2F10E0282F30E0442342
:1029F00029F02C583A4FF901249130E0F6E0CF9FAE
:102A0000C0011124EFEFF0E0BF010E94202FAB01C5
:102A10008C2F90E0880F991FA5E5A49FB001A59F7A
:102A2000700D1124861B970B982F990F980FBF01DB
:102A3000601B710B629FD001639FB00D729FB00D40
:102A400011248B2F9D9FB0011124672F7727EF0151
:102A5000C61BD70BBE01629FE001639FD00D729F22
:102A6000D00D11247F01E91AF108E09EB001E19E2A
:102A7000700DF09E700D1124672F7727E61BF70B62
:102A8000E29F8001E39F100DF29F100D1124E12FB2
:102A9000722F4230510599F048F44115510569F003
:102AA0004130510581F0EB2F8D2F07C04430510587
:102AB00069F080F046305105B1F76E2F8DCFE22FCF
:102AC0007B2F812FFACFE22F7D2FF7CFEB2F822F95
:102AD000712FF3CF7B2F822FED2FEFCF41E00C949E
:102AE000D91430E020E0869F212D969F200D311DC6
:102AF0001124C9010895AC018230910508F40895AC
:102B00009FEF413E8EE1580740F49A0195E03695DB
:102B100027959A95E1F798E0920F61E0E62FE90F8B
:102B2000FF27FF1F9F0135952795822F229FF001D8
:102B3000239FF00DF00D11244E175F0738F49FEF1F
:102B4000920F961758F78FEF860F08952F3FE9F3EE
:102B500061E0620FF6CFE82F86FDE0952E2F2F70F3
:102B600086FD2F5FE695E695E695E670F0E0EF507E
:102B7000FD4F9181929F902D212D112492959F7050
:102B80002295207F922B2081920F87FD919580E8DE
:102B9000890F0895622F0895E42FF0E0EE0FFF1FD4
:102BA000E25AFE4F6081621B0895E42FF0E0EE0FC1
:102BB000FF1FE15AFE4F6081621B0895322F50E0E3
:102BC000FA01EE0FFF1FE15AFE4F9081905297FDE0
:102BD0009195440F551FFA01E25AFE4F2081231BA5
:102BE000330B290F311D97FD3A95620F0895EF922F
:102BF0000F93972F23E0029FB001112475956795DD
:102C00006E0D792F0F91EF9008950F93CF93DF936F
:102C1000D72FC82F47FD419588E390E0841B910989
:102C200047FD9395889FB001899F700D700D112409
:102C3000229FC001239F900D900D1124860F971F96
:102C40000E947B15982F990F890F682F600F7D2F99
:102C50008C2FDF91CF910F9108950F931F93522FD7
:102C600010E0F801EE0FFF1FE15AFE4FA081A052C5
:102C7000BB0B9D015203F001539FF00D1124000F77
:102C8000111FD801A25ABE4F0C910057110B4003DF
:102C90009001419F300D11242E0F3F1F37FF02C0BE
:102CA00021583F4F220F232F221F330B620F1F91FA
:102CB0000F9108950F931F93522F10E0F801EE0F1C
:102CC000FF1FE15AFE4FA081A052BB0B9D01520392
:102CD000F001539FF00D1124000F111FD801A25ACB
:102CE000BE4F0C910057110B40039001419F300DD6
:102CF00011242E0F3F1F37FF02C0215C3F4F96E08B
:102D0000359527959A95E1F7620F1F910F910895D8
:102D1000FC019B01AC0197FF04C044275527481BC9
:102D2000590BBA01620F731F37FD0FC0241B350BFF
:102D3000C901A5E0880F991FAA95E1F70E94342FD9
:102D400080E2861BF7FD81950895CB0165E0880F31
:102D5000991F6A95E1F7BA01621B730B0E94342F29
:102D600080E6EFCFEF920F93CF93DF93D72FC82F4B
:102D7000C9010E19009729F480E857FD05C080E0CD
:102D800003C0BA010E948816602F681B7D2F8C2F0C
:102D9000DF91CF910F91EF90089546E050E06CE104
:102DA00070E088E394E00E9407301092AF0308952A
:102DB0000F93CF93DF93D72FC82FC901009729F422
:102DC00080E857FD05C080E003C0BA010E94881664
:102DD000602F680F7D2F8C2FDF91CF910F91089579
:102DE0000C946E150C94CD16E8E3F4E081E1808339
:102DF00080916B0290916C02A0916D02818392830D
:102E0000A3838FE784838FEF85830C94CD16E091A5
:102E1000FF02F09100030994E091FB02F091FC02A3
:102E200009945F926F927F928F929F92AF92BF921E
:102E3000CF92DF92EF92FF920F931F93CF93DF9386
:102E40005C014B01FC01C08181E1C89FC02D1124B0
:102E500011E11C0FF12E133510F032E5F32E6091C5
:102E60003C04669580913E0490913F040E94711548
:102E7000582ED0E0CF15A0F081E0123508F080E0A8
:102E8000DF91CF911F910F91FF90EF90DF90CF9046
:102E9000BF90AF909F908F907F906F905F900895BC
:102EA000FE01EE5FFD4F8081F50191818923C9F11B
:102EB000CE01880F991F8C5F9E4FFC01E65AFF4F91
:102EC0002081422F4057550B6A01855A9F4FFC01C4
:102ED0008081282F2052330B3901449F9001459F58
:102EE000300D300D1124669CC001679C900D900D33
:102EF0001124820F931F0E947B15082F60913904C3
:102F000070913A0480913B04E52C9301A601F401F1
:102F100009950E94F016462F282F672FCE010E9498
:102F20000C172196A7CF67EF75E10C94111762EB90
:102F300076E10C941117AF92BF92CF92DF92EF928D
:102F4000FF920F931F93CF93DF936C017B01FC01E2
:102F5000C08181E1C89FC02D112411E11C0FB12E49
:102F6000133510F032E5B32E60913C0466958091E4
:102F70003E0490913F040E947115A82ED0E0CB151D
:102F800078F081E0123508F080E0DF91CF911F9159
:102F90000F91FF90EF90DF90CF90BF90AF9008958A
:102FA000FE01EE5FFD4F8081F6019181892311F1D1
:102FB000CE01880F991F8C5F9E4FFC01E55AFF4F91
:102FC00020812052330B865A9F4FFC01408140578D
:102FD000550B6091390470913A0480913B040A2D9D
:102FE000F70109950E94F016462F282F672FCE0172
:102FF0000E940C172196C3CF65E076E10C949B17D5
:1030000068ED76E10C949B17BF92CF92DF92EF921E
:10301000FF920F931F93CF93DF937C018B01FC01F1
:10302000C08181E1C89FC02D112491E1D92EDC0E11
:10303000CD2CF2E5FD1510F482E5C82E60913C041C
:103040006695669521E0620F08F46FEF80913E046B
:1030500090913F040E947115B82ED0E0CC1578F005
:1030600081E091E59D1508F480E0DF91CF911F91FB
:103070000F91FF90EF90DF90CF90BF900895FE01E9
:10308000EE5FFD4F8081F7019181892391F060917E
:10309000390470913A0480913B042B2D4C2FF80198
:1030A00009950E94F016462F282F672FCE010E9407
:1030B0000C172196D3CF6AEC75E10C9404186CECD4
:1030C00075E10C94041865ED75E10C9404186EED2F
:1030D00075E10C9404187F928F929F92AF92BF92E9
:1030E000CF92DF92EF92FF920F931F93CF93DF93D4
:1030F0005C016B01FC01C08181E1C89FC02D1124DE
:1031000011E11C0F912E133510F032E5932E6091D2
:103110003C046695669580913E0490913F040E9420
:103120007115F82E80E48F0D0E94AB1590E8892E62
:10313000880E8F2D0E94AB1520E8722E780ED0E0FD
:10314000C91590F081E0123508F080E0DF91CF9151
:103150001F910F91FF90EF90DF90CF90BF90AF90B5
:103160009F908F907F900895FE01EE5FFD4F8081CC
:10317000F50191818923A1F06091390470913A049D
:1031800080913B04EF2C0C2F272D482DF60109953B
:103190000E94F016462F282F672FCE010E940C1791
:1031A0002196CECF6DE276E10C946B186AE576E15C
:1031B0000C946B18BF92CF92DF92EF92FF920F9315
:1031C0001F93CF93DF937C01FC01C08181E1C89FF5
:1031D000C02D112411E11C0F012F133508F002E559
:1031E0006091390470913A0480913B040E94F0167A
:1031F000D62EC72EB82ED0E0C01770F081E0123561
:1032000008F080E0DF91CF911F910F91FF90EF9038
:10321000DF90CF90BF900895FE01EE5FFD4F80815B
:10322000F7019181892331F02B2D4D2D6C2DCE018D
:103230000E940C172196E0CFBF92CF92DF92EF92BF
:10324000FF920F931F93CF93DF938C01FC01C081FA
:1032500081E1C89FC02D112491E1F92EFC0EEF2CC5
:10326000F2E5FF1510F482E5E82ED0903904D091F4
:103270003A04C0903B0460913C046695669566955F
:1032800080913E0490913F040E9471150E94AB15FD
:10329000805887FD8195880F282F3C2D239F212D55
:1032A0001124822F6D2D7D2F0E94F016D62EC72E51
:1032B000B82ED0E0CE1578F081E021E52F1508F486
:1032C00080E0DF91CF911F910F91FF90EF90DF9001
:1032D000CF90BF900895FE01EE5FFD4F8081F80111
:1032E0009181892331F02B2D4D2D6C2DCE010E9423
:1032F0000C172196DFCFDF92EF92FF920F931F936F
:10330000CF93DF938C01FC01EE5FFD4F808168233A
:1033100081F1D0903A04D0913B04C0913904EC2E55
:10332000F12C0E94C32F282FC7018C549F4F68E6B1
:1033300071E00E94342F8E199F0997FD0396959591
:1033400087959595879523706C2F289F600D112484
:103350007D2D8D2F0E94F016462F282F672FC80134
:10336000DF91CF911F910F91FF90EF90DF900C9420
:103370000C17DF91CF911F910F91FF90EF90DF908D
:103380000895DF92EF92FF920F931F93CF93DF93F5
:103390008C01FC01C281C11125C060913C0420E177
:1033A000620F08F46FEF80913E0490913F040E94F9
:1033B00071156AE070E00E94202F892B51F40E9461
:1033C000C32F62E570E00E94342FF80161810E94F2
:1033D0007B198C2FDF91CF911F910F91FF90EF9070
:1033E000DF900895C08181E1C89FC02D112481E143
:1033F000D82EDC0E8D2DF2E5FD1508F482E5D0E027
:10340000E82EF12CCE15DF0534F0C1E0F1E5FD1515
:1034100000F7C0E0DECFF8016181CE010E947B1988
:103420002196F0CFE091FD02F091FE0209940C94F8
:103430003110CF93C82F80915C028C1323C09091E0
:103440003804937020915D0230E081E092171306FA
:1034500009F480E0817080935B0280913D0490913B
:103460005A02981739F080935A0240E060E080E0F9
:103470000E94121ACE3088F4EC2FF0E0E456FF4C94
:103480000C946A2F81E0E6CF80915B02882359F08B
:1034900040E060E080E00E94121A80E004C089E50C
:1034A00092E00E94DA18909159029F5F909359021E
:1034B00081110CC082E08093580280915B028111DF
:1034C00005C0C11103C083E080935802CF910895D5
:1034D00089E592E00E941C19E6CF89E592E00E94FE
:1034E0005B18E1CF89E592E00E945F18DCCF89E5A7
:1034F00092E00E946318D7CF89E592E00E94671896
:10350000D2CF89E592E00E949317CDCF89E592E072
:103510000E94FC17C8CF89E592E00E940018C3CF33
:1035200089E592E00E949717BECF89E592E00E945C
:10353000D218B9CF89E592E00E94D618B4CF89E5B8
:1035400092E00E94C119AFCF089508950E94A41A75
:103550000C94A51A08950895CF93DF93FC01C081C0
:1035600081E1C89FC02D1124DFEEDC0FC33508F0C8
:10357000C2E56C2F8D2F0E94AA1A6C2F8D2FDF9120
:10358000CF910C94AB1ACF930E9439276093B0036C
:103590007093B1038093B2039093B3032091B4036B
:1035A000C0E0211108C020913804C22FC37019F067
:1035B000C22FC695C695209158022130B1F0222322
:1035C00031F02230F1F0233039F1CF91089510928B
:1035D000590260933E0470933F048093400490939B
:1035E000410481E080935802F0CF8C2F0E94191A79
:1035F000CC2359F30E94A61A89E592E0CF910C944E
:10360000AC1AC0935C0280913804837080935D0291
:103610000E94071783E0E6CF8091AF0381110E94DB
:10362000CD1660913E0470913F04809140049091CA
:1036300041040E945427603171058105910528F2EB
:1036400010925802C2CFE091F902F091FA02099566
:103650000E945B0F811104C00E94FF0F0E94F416AC
:1036600046E050E06CE170E088E394E00E94E92FCE
:103670001092AF03809138048C7F11F40C94F416EF
:103680000895CF93C82F882391F08091B4038111BE
:103690000EC00E94191A10925C0280913804837047
:1036A00080935D020E94071783E080935802C093C5
:1036B000B403CF910895E8E3F4E0908121E09227EC
:1036C0009083109258029091AF03892B8093AF039F
:1036D000089581E00C945B1B80913804837011F491
:1036E00010925802809138048C7F81608093380456
:1036F000089580913804837011F0109258028091DF
:1037000038048C7F80933804089590913804937026
:1037100061F081110BC094609093380410925802AC
:103720008091AF03862B8093AF0308958E3010F005
:103730009463F2CF880F880F982BEECF60E00C9443
:10374000851B61E00C94851B8091380486958695D5
:103750000895682F909138049695969581E0890F89
:103760008E3008F081E00C94851B81E00C94A91B3D
:10377000682F90913804969596958FEF890F09F4EC
:103780008DE00C94851B81E00C94B81B909138045B
:10379000937059F08093390460933A0440933B044A
:1037A0008091AF03822B8093AF03089520E00C94A7
:1037B000C61B80913904089580913A040895809140
:1037C0003B040895A8E3B4E01196EC911197F0E062
:1037D000282F13964C91139712966C91CF0108964F
:1037E0000C94C61B81E00C94E21BE8E3F4E09181A9
:1037F000282F43816281E92FE850FF0BCF010C9401
:10380000C61B81E00C94F51BE8E3F4E0628120E143
:10381000620F08F46FEF9181282F4381892F90E088
:103820000C94C61B81E00C94041CE8E3F4E0628174
:1038300020E1621B08F460E09181282F4381892FE9
:1038400090E00C94C61B81E00C94151CE8E3F4E0B6
:10385000438120E1420F08F44FEF9181282F6281CC
:10386000892F90E00C94C61B81E00C94261CE8E3A1
:10387000F4E0438120E1421B08F440E09181282FCD
:103880006281892F90E00C94C61B81E00C94371C58
:1038900080933C048091AF03862B8093AF030895FF
:1038A00060E00C94481C80913C04089520913C04F5
:1038B00030E1230F08F42FEF682F822F0C94481C5F
:1038C00081E00C94561C20913C0430E1231B08F449
:1038D00020E0682F822F0C94481C81E00C94631C1C
:1038E00060E080E50E94111E61E08FE50C94111EDE
:1038F000CF930E94AE2460E080E50E94D81C60E077
:103900008FE50E94D81CC0E021E041E061E08C2FEF
:103910000E948B1DCF5FC235B9F760E080E50E9441
:10392000461E61E08FE5CF910C94461E6093C20560
:103930004093C30524E630E042E050E062EC75E0DD
:10394000880F0E945D2521E0892B09F020E0822F5D
:103950000895EF92FF921F93CF93DF937B01182F6F
:10396000110FD0E0C0E0C093C205D701AC0FBD1F5E
:10397000E3ECF5E08D91819385E0E33DF807D1F725
:1039800024E630E041E150E062EC75E0812F0E94D6
:103990005D25892B59F46096C03CD10521F781E063
:1039A000DF91CF911F91FF90EF90089580E0F8CFC5
:1039B0001F93CF93DF93C82FD62F45EC6EEF0E9455
:1039C000961C40E06DEF8C2F0E94961C10E040E0AA
:1039D000612F8C2F0E94961C1F5F1831C1F745EC98
:1039E0006EEF8C2F0E94961C41E06DEF8C2F0E9491
:1039F000961C10E040E0612F8C2F0E94961C1F5FE8
:103A0000103CC1F745EC6EEF8C2F0E94961C43E0F2
:103A10006DEF8C2F0E94961C40E06FE08C2F0E946F
:103A2000961C40E060E18C2F0E94961C4FEF61E0F5
:103A30008C2F0E94961C80E4D89FA0011124416025
:103A400060E08C2F0E94961C8FE39CE90197F1F7B0
:103A500000C00000DF91CF911F910895FF920F9356
:103A60001F93CF93DF9300D000D0CDB7DEB7F62EF3
:103A7000042F122F8235910550F5880F991F880F5A
:103A8000991FBC0164557F4F44E050E0CE01019680
:103A90000E94D32F89818370AA81E82FF0E020EC67
:103AA000829FC00111248E5B9B4FA80FB92FB11DBF
:103AB000FC92AB81A80FB92FB11D0C932C81820F02
:103AC000911DDC011C93E951FC4F81E080830F9034
:103AD0000F900F900F90DF91CF911F910F91FF905A
:103AE0000895FF920F931F93CF93DF93182F062F04
:103AF000F42ED0E0C0E02F2D402F612FCE010E9488
:103B00002E1D2196C235D105B1F7DF91CF911F91BE
:103B10000F91FF900895FF920F931F93CF93DF9320
:103B200000D000D0CDB7DEB7F62E042F122F24E040
:103B3000829FB001112464557F4F44E050E0CE01D4
:103B400001960E94D32F9A81AB81BA2FB695B69574
:103B5000B6956C81762F769576957695A770677079
:103B6000E92FE695E695E695F0E0977021E030E0E4
:103B700001C0220F9A95EAF78981982F937048E146
:103B8000949FE00DF11D1124E954FC4FFF20F1F149
:103B90009081922B90838370482F50E0E8E18E9FB4
:103BA000C001112489549C4FFC01EB0FF11D908141
:103BB00021E030E001C0220FAA95EAF7002359F175
:103BC000292B208388E1849FF001859FF00D11242B
:103BD000E954FC4FE70FF11D208181E090E001C026
:103BE000880F6A95EAF71123C9F0822B80834B5422
:103BF0005C4F81E0FA0180830F900F900F900F903F
:103C0000DF91CF911F910F91FF900895922F909582
:103C100020819223BFCF20952923D3CF8095822363
:103C2000E5CFEF92FF920F931F93CF93DF93D82F9F
:103C3000C62F062F10E0C80189519C4F7C01FC0162
:103C400080818823D1F045EC6EEF8D2F0E94961C69
:103C500041E06DEF8D2F0E94961CF0ECCF9FB001DC
:103C600011246E5B7B4F8D2F0E94A91C811105C012
:103C7000F801EB54FC4F81E08083F7011082DF9163
:103C8000CF911F910F91FF90EF900895EF92FF92C7
:103C90000F931F93CF93DF93E82EC62F062F10E0CC
:103CA0000B541C4FF80180818823D1F045EC6EEF56
:103CB0008E2D0E94961C40E06DEF8E2D0E94961C6A
:103CC000F8E1CF9FE0011124C954DC4FF12C499158
:103CD0006F2D8E2D0E94961CF39488E1F812F7CF79
:103CE000F8011082DF91CF911F910F91FF90EF901B
:103CF0000895FA01811101C0FB0109940F931F93EC
:103D0000CF938C01FB01C281CC2309F48FC00E94A8
:103D1000740E82720A3CFCE51F0709F472C060F55C
:103D2000053CECE51E0709F458C080F4033C9CE513
:103D3000190709F448C008F04BC0023C1C4509F4BF
:103D40003FC08C2FCF911F910F910895073C9CE5A8
:103D5000190709F44CC008F445C0083CFCE51F07EE
:103D600009F44AC045E45CE164E37CE1093C1C459C
:103D700041F70E94791E1EC00F3CECE51E0709F4B6
:103D800053C080F40C3C9CE5190709F444C0F0F1E1
:103D90000D3CFCE51F0709F443C00E3C1C4589F6A9
:103DA00082E03FC0063D9CE5190730F489E0013D03
:103DB0001C45B8F1C0E0C5CF0D351D45D9F3C1CFC5
:103DC0000E94691BF7CF43EC5BE165EB7BE1D1CF50
:103DD00045EB5BE163EC7BE1CCCF41E05CE162EF82
:103DE0007BE1C7CF42EF5BE161E07CE1C2CF43E220
:103DF0005CE162E17CE1BDCF42E15CE163E27CE158
:103E0000B8CF44E35CE165E47CE1B3CF4DE65CE12F
:103E100060E67CE1AECF40E65CE16DE67CE1A9CFF7
:103E200081E00E94A11BC6CF84E0FBCFC1E089CF17
:103E300083E290E00E94F92F823289F484E290E0DC
:103E40000E94F92F823059F485E290E00E94F92F08
:103E500091E0823109F090E0892F8170089580E02F
:103E6000FCCFCF93C82F6FEF811162E283E290E025
:103E70000E9417306FEFC11162E084E290E00E946F
:103E800017306FEFC11162E185E290E0CF910C94A1
:103E90001730089586E290E00E94F92F682F70E0B5
:103EA00090E080E0089586E290E00C94173080E086
:103EB0000E94311F60E070E0CB010E94531F0E94FE
:103EC00073220E945F2381E00C94311F0E94491FDE
:103ED0000E94181F811102C00C94571F0895CF93A0
:103EE000FB01C281CC2309F19C0122513F452031C5
:103EF000310520F582510E946F23C0E08C2FCF91B5
:103F0000089581E00E94280A43E062E081E00E9477
:103F10000005F3CF81E00E94330A43E062E081E0D4
:103F20000E940005EBCF82E0F6CF8031FFE59F07CE
:103F300089F381319F45B9F3C1E0E0CF8031EFE5EE
:103F40009E07F9F281319F45C9F682E0DBCF2FEF62
:103F5000FC0120830895CF93DF93EC0188818138A1
:103F6000A9F028F4803871F0DF91CF91089582385C
:103F700081F08338C9F70E94D91B89830E94DC1B1A
:103F80008A83F2CF0E94DF1B8983EECF0E94A41B9D
:103F9000FBCF0E94531CF8CFCF93DF93EC018881B5
:103FA0008138F1F028F4803871F0DF91CF910895D5
:103FB000823821F18338C9F70E94DF1B9981482F8D
:103FC0006A81892F08C0D9810E94DC1BC82F0E94FA
:103FD000D91B4D2F6C2F90E0DF91CF910C94D61B05
:103FE00089810E949E1B8981811104C0DF91CF913C
:103FF0000C94791BDF91CF910C946C1B8981DF911C
:10400000CF910C94501CEF92FF920F931F93CF937C
:10401000DF93EC01062FDC01ED91CD01E150E3319E
:1040200008F0ADC0F0E0E655FF4C0C946A2F198201
:1040300089E08A83602FCE01DF91CF911F910F918C
:10404000FF90EF900C942F288981823069F08330A3
:1040500071F08130D9F40E9439270E94702F6A8351
:104060007B838C839D83E6CF0E944A1FF6CF7E011F
:1040700010E0812F0E943A13F701928383831F5F20
:10408000F2E0EF0EF11C1630A1F7D4CF602FCE0175
:104090000E94A71FCFCF89818230C1F76A817B81BF
:1040A0008C819D810E94702F0E94531FC3CF4B8132
:1040B0006A8189810E9445229827892798279D83B4
:1040C0008C83B8CF2C813D813227232732274B8127
:1040D0006A8189810E945E22ADCF0E947322AACF9D
:1040E0000E94CC1FA7CF0E94AB1FA4CF0E94F21644
:1040F000A1CF0E94082389839DCF0E940A2398277D
:10410000892798279A83898395CF6B8170E089816D
:104110009A81AE014C5F5F4F9827892798270E94AC
:104120000D2388CF6B8170E089819A81AE014C5F4D
:104130005F4F9827892798270E9434237BCF0E94BE
:104140005F2378CF0E943322D6CF6B8170E08981C4
:104150009A81AE014C5F5F4F9827892798270E946C
:10416000AB2268CF6B8170E089819A81AE014C5F90
:104170005F4F9827892798270E94D1225BCF8FEF26
:10418000888358CFCF93DF93EC01FB018281882392
:1041900009F420C1C330FDE5DF07C8F5CA3F9CE53F
:1041A000D90730F49E0122503C452431310598F561
:1041B0000E946E0F90931F0480931E04C031FCE593
:1041C000DF0709F4E0C008F061C0C8309CE5D907FA
:1041D00009F4CBC088F5C430FCE5DF0709F4B3C0AF
:1041E000E8F4C2309CE5D90709F4A7C080911E0409
:1041F0008260C330DC4509F4A3C080911E04909115
:104200001F040E947C0F0E94AF0980E004C0C136E9
:10421000EDE5DE0769F2DF91CF91089580911E04EC
:104220008061C630FCE5DF0709F48AC008F48FC05E
:1042300080911E04806284C080911E048D7FCC30EA
:104240009CE5D90709F47CC070F480911E048C6051
:10425000CA30FCE5DF0709F473C008F48AC0809116
:104260001E048E7F6DC080911E04877FCE309CE53A
:10427000D90709F465C080911E048B7FCF30DC45DF
:1042800008F45EC080911E048F7E5AC0CC3FFCE5CE
:10429000DF0709F474C040F5C4319CE5D90709F47F
:1042A0008AC058F4C231FCE5DF0709F474C008F491
:1042B0006EC080911E04837F43C0CA3F9CE5D9072E
:1042C00009F449C008F04DC0C531DC4509F095CF6F
:1042D00080911E0482FB992790F921E0922790FBA0
:1042E00082F990FB83F92CC0C1158DE5D80709F43C
:1042F00058C088F480911F048360CE3FECE5DE0750
:1043000069F180911F048D7FCF3FDC4538F18091AA
:104310001F048C7F23C0C2308DE5D80709F458C034
:1043200008F452C0C136DD4509F067CF90911E04F4
:10433000892F8F7E94FF806103C080911E0481606D
:1043400080931E045ACF80911E048460F9CF80911F
:104350001E048860F5CF80911F04816080931F0444
:104360004CCF80911F048260F9CF80911E0480643D
:10437000E7CF0E94AF0980911E048068E1CF809151
:104380001F048E7FEBCF80911E048F7DD9CF80914B
:104390001E048F7BD5CF0E94AF0980911E048F77BA
:1043A000CFCF80911F04982F909591708E7F892B8D
:1043B00090FB81F9D3CF0E94AF0990911E04892F01
:1043C00097FB87F98058BCCF81E00E94011015CF80
:1043D00080E0FBCF81E01FCF81E0089581E0089568
:1043E0000C94EE211092EC031092EB030895CF92FF
:1043F000DF92EF92FF92CF93C82F8091EB039091C1
:10440000EC03843F21E0920768F401969093EC035B
:104410008093EB030A9721F1CF91FF90EF90DF900B
:10442000CF90089540E061E080E00E9453138093B4
:10443000EA03C82ED12CF12CE12C9091E9038913C9
:1044400002C0CC2349F3682F80E00E943A04C701E0
:10445000B6010E94F0218091EA038093E903DCCF4A
:1044600041E0C1E0E0CF84E0089550E0440F551FE3
:104470009EE1699F400D511D112494EB899F400DD1
:10448000511D1124CA01879608950F931F93CF934E
:10449000DF930E9435228C010E94F92FC82FD0E0B3
:1044A000DC2FCC27C80101960E94F92F9E01282BF2
:1044B000C901DF91CF911F910F9108950F931F9321
:1044C000CF93DF93122F032F0E943522EC01602F30
:1044D0000E941730612FCE010196DF91CF911F917D
:1044E0000F910C941730AF92BF92CF92DF92EF9260
:1044F000FF921F93CF93DF9384EFC82E81E0D82ED5
:10450000D0E07601C0E014C0F50125913491412F2F
:104510006C2F8D2F0E945E2282E0A80EB11C1F5FBF
:104520001F3091F78EE1E80EF11CCF5FC63019F015
:10453000570110E0E9CFDF5F84EBC80ED11CD43007
:1045400001F7DF91CF911F91FF90EF90DF90CF9017
:10455000BF90AF900895EF92FF920F931F93CF9368
:10456000DF93EC018A017C01E60EF71ECE018796EF
:10457000CE15DF0539F4DF91CF911F910F91FF9098
:10458000EF900895C03D22E0D20740F40E94F92F39
:10459000F80180830F5F1F4F2196E8CFF80110824A
:1045A000F9CFCF92DF92EF92FF920F931F93CF93A9
:1045B000DF937C016A018C01060F171FEC01CE010D
:1045C0008796C017D10749F4DF91CF911F910F91C2
:1045D000FF90EF90DF90CF900895C03D22E0D2078A
:1045E00040F4FE01EE19FF09EC0DFD1D60810E94F3
:1045F00017302196E4CF462F843038F4763028F4F3
:104600006F3018F4672F0C94452290E080E00895F5
:1046100080E1089589E091E00895EF92FF920F9371
:104620001F93CF93DF93EC018A017C01E60EF71E06
:10463000CE0189509D4FCE15DF0539F4DF91CF9122
:104640001F910F91FF90EF900895C93021E0D2079C
:1046500040F40E94F92FF80180830F5F1F4F2196CD
:10466000E7CFF8011082F9CFCF92DF92EF92FF925D
:104670000F931F93CF93DF937C016A018C01060F88
:10468000171FEC01CE0189509D4FC017D10749F487
:10469000DF91CF911F910F91FF90EF90DF90CF901E
:1046A0000895C93021E0D20740F4FE01EE19FF0958
:1046B000EC0DFD1D60810E9417302196E3CFCF9352
:1046C000DF93C7EFD2E060E0CE010E941730219661
:1046D000C11584E0D807B9F7DF91CF910895DF9233
:1046E000EF92FF920F931F93CF93DF9300D000D0F0
:1046F000CDB7DEB7F82E8FE08F1540F08FEF93E047
:104700000E94F92F07EF12E08823C1F00F900F905D
:104710000F900F90DF91CF911F910F91FF90EF902D
:10472000DF900895011584E0180781F3C8010E9405
:10473000F92F811101C0FA940F5F1F4FF110F2CFD2
:1047400019821A821B821C82DD24D39478018FEF98
:10475000E81AF80AC8010E94F92F89831A8288236F
:10476000A9F29FEF980F933078F48A83D9820E5F75
:104770001F4FC7010E94F92F8B83882339F2CE0186
:1047800001960E946706E2CF8701F9CFCF93DF93AE
:10479000EB0186319C4511F50E94740E9A81992394
:1047A00099F08A7A91E009F490E09093ED038111F9
:1047B00009C089E20E944F0E0E94C40E80E0DF9182
:1047C000CF91089585E3F6CF8091ED03811104C068
:1047D00089E20E94560EF0CF85E3FBCF81E0EFCF58
:1047E0000F931F93CF93DF93C42FD22FFC018281AD
:1047F0008823C9F04093F0030E942D279093EF0384
:104800008093EE0380E28C0F883008F050C0C770B0
:1048100081E001C0880FCA95EAF7DF91CF911F911F
:104820000F910C944A071091F003141335C0809136
:10483000EE039091EF030E944527883C910560F5B7
:10484000C0E2CD0F1D17B9F080E2810F883040F42F
:10485000177081E001C0880F1A95EAF70E9451078E
:10486000C83048F481E09D2F977001C0880F9A9559
:10487000EAF70E944A07802F0E944207C830B8F426
:10488000D77081E001C0880FDA95EAF7DF91CF9108
:104890001F910F910C94510780E28C0F883038F4EF
:1048A000C77081E001C0880FCA95EAF7EFCFDF91AA
:1048B000CF911F910F9108950F939C01CB01233F3E
:1048C0004CE5340759F1A8F4283DFCE53F0701F118
:1048D000293D4CE53407D1F1273D3C4591F406E2F2
:1048E00021EE41EE67ED7CE50E94F02380E00F9120
:1048F0000895253FFCE53F07E9F0B0F0263F3C4531
:10490000F9F0FC018281882339F11092F003EFCF96
:1049100007E225EE45EE68ED7CE5E6CF06E221EE06
:1049200040EE63EF7CE5E0CF07E225EE44EE64EF76
:104930007CE5DACF06E221EE42EE65EF7CE5D4CFEE
:1049400007E225EE46EE66EF7CE5CECF08E221E0F9
:1049500045EE69ED7CE5C8CF81E0C9CF1092B90082
:104960008CE08093B80008959F92AF92BF92CF924F
:10497000DF92EF92FF920F931F93CF93DF93B82EA6
:10498000EB010E942D276C01EE24E394F12CC4313D
:10499000D10560F025E0E22EF12CCF3FDC0731F0AD
:1049A000CE0164E170E00E94202F7B0184EAA82EF2
:1049B00094E8992E1092BC00A092BC000E942D2772
:1049C0008C018091BC0087FF0DC08091B900887F69
:1049D000883039F18091B900887F803111F10FEF73
:1049E0001FEF09C00E942D27801B910B8E159F057C
:1049F00040F30EEF1FEFCF3FDC07E1F2C6010E944C
:104A000045278C179D07B0F2C801DF91CF911F9108
:104A10000F91FF90EF90DF90CF90BF90AF909F905D
:104A20000895B092BB009092BC000E942D278C018B
:104A30008091BC0087FF0AC08091B900887F8831CF
:104A400011F0803461F610E000E0DECF0E942D27E7
:104A5000801B910B8E159F0558F3CBCF0F931F939F
:104A6000CF93DF93EB018093BB0084E88093BC007D
:104A70000E942D278C018091BC0087FF11C02091DE
:104A8000B900287F81E090E0283211F490E080E0C6
:104A9000919581959109DF91CF911F910F91089583
:104AA000CF3FDC0741F30E942D27801B910B8C1711
:104AB0009D0708F38EEF9FEFEECFCF92DF92EF923C
:104AC000FF920F931F93CF93DF936B018A017901BC
:104AD000B9010E94B424E6010C0D1D1DC017D107B9
:104AE00061F424E92093BC00DF91CF911F910F91D5
:104AF000FF90EF90DF90CF90089597FDF2CFB70130
:104B000089910E942E25EACF909311038093100380
:104B100008959093F6038093F5030895E091F503CB
:104B2000F091F603309721F00190F081E02D099487
:104B300080E00895E091F503F091F603309799F045
:104B400020916A02222359F020911E0427FF07C0FA
:104B5000DC012C9111962C93119726E02C93028066
:104B6000F381E02D099408952091F3033091F4032B
:104B70002817390771F09093F4038093F303E091C1
:104B8000F503F091F603309721F00680F781E02DD0
:104B9000099408952091F1033091F2032817390701
:104BA00071F09093F2038093F103E091F503F0919B
:104BB000F603309721F00084F185E02D09940895E3
:104BC000FC01329680916A02882321F080911E04B4
:104BD0009EE187FF96E080E0915008F408952191CE
:104BE0002223D1F38F5FF8CF662301F120916A026F
:104BF0002223F1F020911E0427FF1AC0462F46956C
:104C0000469546954E3190F4677021E030E002C041
:104C1000220F331F6A95E2F7840F911DFC018281F8
:104C200090E02823392381E0232B69F480E0089564
:104C3000FC01329608962191261721F0E817F90712
:104C4000D1F7F4CF81E008959C01FC0132969FEFEB
:104C500080E04191461751F09F3F19F4411101C086
:104C6000982F8F5F8630A9F79F3F09F40895290F89
:104C7000311D97FD3A95F90162830895FC01329642
:104C800008962191261303C0DF0111971C92E817A3
:104C9000F907B9F70895E62FE695E695E695EE3122
:104CA00068F4E80FF92FF11D677021E030E001C0D2
:104CB000220F6A95EAF78281822B82830895E62F7C
:104CC000E695E695E695EE3170F4E80FF92FF11DC3
:104CD000677021E030E001C0220F6A95EAF7209565
:104CE000828128232283089520916A02222329F0B9
:104CF00020911E0427FD0C944B260C942426209111
:104D00006A02222329F020911E0427FD0C945F26BD
:104D10000C943E26FC01329680916A02882351F061
:104D200080911E0487FF06C08EE1DF011D928A95E7
:104D3000E9F7089586E0F9CF08950C949C26811137
:104D400005C081E08093F7030C949D2682E0FACFA2
:104D500083E08093F7030C949D260C949F2681E0BA
:104D60008093F7030C949D260C94AF2608958091B0
:104D7000DE05843031F10E9416051092F80388E1B7
:104D800090E020E40FB6F894A895809360000FBEE1
:104D90002093600083B7817F846083BF83B7816085
:104DA00083BF7894889583B78E7F83BF0FB6F894BE
:104DB000A8958091600088618093600010926000E7
:104DC0000FBE089508950895CF930E94E2260E9491
:104DD00031140E94E326C0E08C2F0E943A13892BE5
:104DE00031F4CF5FC630C1F780E0CF91089581E004
:104DF000FCCF0E94AF090C9490051F921FB61F9222
:104E000011248F939F93AF93BF938091F8038111E7
:104E100013C08091D6059091D705A091D805B09187
:104E2000D9054196A11DB11D8093D6059093D70554
:104E3000A093D805B093D905BF91AF919F918F9161
:104E40001F901FBE1F90189582E084BD93E095BD12
:104E50009AEF97BD80936E0008952FB7F8948091D4
:104E6000D6059091D705A091D805B091D9052FBF4F
:104E700008952FB7F8946091D6057091D705809169
:104E8000D8059091D9052FBF08959C014FB7F8948C
:104E90008091D6059091D705A091D805B091D905FC
:104EA0004FBF821B930B0895CF92DF92EF92FF9238
:104EB0002FB7F894C090D605D090D705E090D805CC
:104EC000F090D9052FBFA7019601261B370B480B81
:104ED000590BCA01B901FF90EF90DF90CF90089570
:104EE00078941F921FB61F9211248F939F93AF93B4
:104EF000BF938091D6059091D705A091D805B09128
:104F0000D9050196A11DB11D8093D6059093D705B3
:104F1000A093D805B093D905BF91AF919F918F9180
:104F20001F901FBE1F90189581E08093E00080E2E3
:104F30008093D8001092C9008FE19EE40197F1F7A9
:104F400000C0000087E090EBDC018093E7059093C0
:104F5000E805A093E905B093EA0588E19CE00FB667
:104F6000F894A895809360000FBE90936000FFCFE7
:104F700080911C0408950895CF93DF93EC018091F4
:104F80006A028823B1F180911E0487FF32C060E27B
:104F900084E08093E9008FEF9091E800815095FDC7
:104FA00006C095ED9A95F1F700008111F5CF80913B
:104FB000E80085FF1BC080916A0270E050E040E08D
:104FC000811104C050E040E068E070E0CE010E9432
:104FD000402A8091E8008E778093E80080E2FE010D
:104FE000ACEFB3E001900D928A95E1F7DF91CF919C
:104FF000089568E081E0CDCF8093F9037093FB03BF
:105000006093FA038091DE058430F9F48093E9001F
:105010008FEF9091E800815095FD06C095ED9A952F
:10502000F1F700008111F5CF8091E80085FF0DC0F8
:1050300050E040E063E070E089EF93E00E94402A96
:105040008091E8008E778093E8000895BC0184E0A9
:105050000C94FC27BC0183E00C94FC270895CF93AB
:10506000FC01603221F58091DE05843001F5C091AC
:10507000E900CF702091EC00922F917020FD90E814
:10508000C92B82E08093E9008091E80080FF0CC08A
:1050900050E040E060E270E0CF010E94402A809141
:1050A000E8008E778093E800CF70C093E900CF913D
:1050B00008958091DD05811109C00E941F2C0E9476
:1050C0007C2C8091E20084608093E200089510922D
:1050D000DD0508950C94AF266091DA0581E0611139
:1050E00001C080E00C94A8269091DE0581E0943008
:1050F00009F080E06091DA050C94AD2642E061ECA5
:1051000081E00E949B2B42E261EC84E00E949B2B99
:1051100042E261EC82E00E949B2B42E260EC83E081
:105120000E949B2B9091DE0581E0943009F080E095
:105130006091DA050C949F268091E005833009F494
:1051400062C030F48130D9F1823009F49EC00895F4
:105150008A3009F48AC08B3009F470C0893009F0B4
:1051600051C08091DF05813209F04CC08091E30588
:105170009091E405009719F0029709F043C08091DF
:10518000E800877F8093E8008091E80082FF36C0C6
:105190009091F3008091F200029731F48091F10038
:1051A000813011F0863021F48091F10080931C044D
:1051B0008091E8008B778093E8000C94CF2B80914E
:1051C000DF05813AF9F48091E800877F8093E80059
:1051D0008091E3059091E405892B61F460E28CEF06
:1051E00093E070E00E94DE2A8091E8008B77809344
:1051F000E800089560E090E080E0F3CF8091DE0564
:105200008111C2CF08958091DF05813AD9F780914D
:10521000E3059091E405892BA9F78091E800877F49
:105220008093E8008091E80080FFFCCF80916A02C3
:105230008093F1008091E8008E77BDCF8091DF05EB
:10524000813201F78091E3059091E405892BD1F635
:105250008091E800877F8093E8000E94CF2B8091A7
:10526000E10580936A020C94AF098091DF058132D9
:1052700049F68091E800877F8093E8000E94CF2B59
:105280008091E20580931D0408958091DF05813AA5
:1052900009F0B8CF8091E800877F8093E800809183
:1052A000E80080FFFCCF80911D04C2CF84B7877FC8
:1052B00084BF0FB6F894A8958091600088618093B0
:1052C0006000109260000FBE80E890E00FB6F89486
:1052D00080936100909361000FBE0C94B4260E94ED
:1052E0001F2C0E947C2CE2EEF0E0808184608083A1
:1052F00078940C94052F8EE592E00C94892580918A
:10530000DE058530A9F48091DE05853011F00C941E
:10531000F9260E94B7268091DC058823A1F30E941C
:10532000E426882381F30E942A2A0E94AF09EBCF4A
:105330000895CF93DF93CDB7DEB7A0970FB6F8945B
:10534000DEBF0FBECDBF8091DE05843009F583E05E
:105350008093E9008091E80082FF1AC08091E80004
:1053600090E085FF09C050E040E060E270E0CE01CF
:1053700001960E948F2A91E08091E8008B778093BC
:10538000E800992329F060E2CE0101960E940320F3
:10539000A0960FB6F894DEBF0FBECDBFDF91CF91C0
:1053A00008950C94D329292F33272330310521F177
:1053B00068F42130310509F443C02230310509F485
:1053C00044C090E080E030E020E026C0213231058A
:1053D00051F122323105A9F76330710590F7FB01D5
:1053E000EE0FFF1FEC5FFC4F208131816F5F7C4F20
:1053F000FB01808190E010C099278130910581F0F8
:10540000009729F00297E9F6E4E7F6E002C0E2EA45
:10541000F6E0849190E09F01FA01318320830895A2
:10542000EEE8F6E0F6CF6330710558F6660F771FA9
:10543000FB01E65FFC4F2081318189E090E0ECCFF9
:1054400082E190E021E037E0E7CF8BE590E026EACB
:1054500036E0E2CF80E189BD82E189BD09B400FE7A
:10546000FDCF8091D8008F7D8093D8008091E0009F
:1054700082608093E0008091E00081FDFCCF089580
:10548000AF92BF92CF92DF92FF920F931F93CF9371
:10549000DF936C01EB018A010E94EE2BF82E811143
:1054A00023C00115110539F0F80180819181C81BD5
:1054B000D90BC80ED91EB12CA12C2097A9F0809130
:1054C000E80085FD22C08091E8008E778093E80097
:1054D00001151105A1F0F80180819181A80EB91E76
:1054E000B182A08285E0F82E8F2DDF91CF911F91A0
:1054F0000F91FF90DF90CF90BF90AF9008950E94E2
:10550000EE2B8823D1F2F82EEFCFF60181916F01B7
:105510008093F1002197FFEFAF1ABF0ACECFAF9271
:10552000BF92CF92DF92FF920F931F93CF93DF939F
:105530006C01EB018A010E94EE2BF82E811123C031
:105540000115110539F0F80180819181C81BD90B33
:10555000C80ED91EB12CA12C2097A9F08091E8008B
:1055600085FD22C08091E8008B778093E8000115CB
:105570001105A1F0F80180819181A80EB91EB182B8
:10558000A08285E0F82E8F2DDF91CF911F910F9192
:10559000FF90DF90CF90BF90AF9008950E94EE2BC8
:1055A0008823D1F2F82EEFCF8091F100F60181939C
:1055B0006F012197FFEFAF1ABF0ACECFFC01809198
:1055C000E5059091E60586179707A0F0611571052E
:1055D00029F49091E8009E779093E80090E061159F
:1055E000710551F4911108C08091E80082FF34C028
:1055F00080E00895BC01F2CF8091DE058823C1F1DF
:105600008530C1F18091E80083FD30C08091E800D1
:1056100082FDEACF8091E80080FFE1CF8091F30026
:105620002091F200382F6115710519F028303105ED
:1056300058F091E02830310509F090E02091E80021
:105640002E772093E800CBCF81918093F1006150B9
:1056500071092F5F3F4FE7CF8091DE05882341F02E
:10566000853041F08091E80083FFBECF81E008954E
:1056700082E0089583E00895FC018091E505909112
:10568000E60586179707A0F06115710529F480914A
:10569000E8008E778093E80090E06115710551F481
:1056A000911108C08091E80082FF35C080E0089524
:1056B000BC01F2CF8091DE058823C9F18530C9F1A4
:1056C0008091E80083FD31C08091E80082FDEACF3F
:1056D0008091E80080FFE1CF8091F3002091F200FB
:1056E000382F6115710519F02830310558F091E017
:1056F0002830310509F090E08091E8008E778093A2
:10570000E800CBCF84918093F1003196615071090C
:105710002F5F3F4FE6CF8091DE05882341F0853033
:1057200041F08091E80083FFBDCF81E0089582E0E1
:10573000089583E00895982F973028F08F70809314
:10574000E90081E008959093E900242F762F50E03E
:10575000981731F07091EC002091ED005091F0001D
:1057600021FD02C09F5FE8CF3091EB003E7F309378
:10577000EB003091ED003D7F3093ED003091EB0078
:1057800031603093EB007093EC002093ED00509368
:10579000F0002091EE0027FDE5CF80E00895809194
:1057A000DF0587FF13C08091E80082FF06C080916B
:1057B000E8008B778093E80004C08091DE058111BA
:1057C000F2CF08958091DE058823D9F38091E80017
:1057D00080FFF8CF8091E8008E77ECCF2091E40035
:1057E0003091E50095E6A9012091EC00822F8170AF
:1057F00020FF06C08091E80080FF06C080E0089589
:105800002091E80022FD1AC08091DE05882389F0EE
:10581000853089F08091EB0085FD0FC02091E40078
:105820003091E50042175307F9F29150E1F684E018
:10583000089582E0089583E0089581E008950E942C
:105840008D2C0E94952CE0EEF0E0808181608083B9
:10585000E8EDF0E080818F77808319BCA7EDB0E0A0
:105860008C918E7F8C9380818F7E80831092DD055A
:1058700008950F931F93CF93DF930E948D2C0E9466
:10588000952CC8EDD0E088818F77888388818068E7
:10589000888388818F7D888319BC1092DE051092E1
:1058A000DA051092DC051092DB0500EE10E0F8013D
:1058B00080818B7F808388818160888342E060E083
:1058C00080E00E949B2BE1EEF0E080818E7F808360
:1058D000E2EEF0E080818160808380818860808357
:1058E000F80180818E7F8083888180618883DF9149
:1058F000CF911F910F910895E8EDF0E080818F7EA8
:105900008083E7EDF0E080818160808384E082BF66
:1059100081E08093DD050C94392CE8EDF0E0808186
:105920008E7F80831092E20008951092DA00109228
:10593000E10008951F920F920FB60F9211242F933A
:105940003F934F935F936F937F938F939F93AF9307
:10595000BF93EF93FF938091E10082FF0BC0809192
:10596000E20082FF07C08091E1008B7F8093E1001D
:105970000E94042F8091DA0080FF19C08091D80026
:1059800080FF15C08091DA008E7F8093DA008091CD
:10599000D90080FF96C080E189BD82E189BD09B44C
:1059A00000FEFDCF81E08093DE050E9459288091A2
:1059B000E10080FF19C08091E20080FF15C0809156
:1059C000E2008E7F8093E2008091E200806180930C
:1059D000E2008091D80080628093D80019BC85E0F5
:1059E0008093DE050E946C288091E10084FF2BC02B
:1059F0008091E20084FF27C080E189BD82E189BDFA
:105A000089B5982F917080FFFBCF8091D8008F7D52
:105A10008093D8008091E1008F7E8093E100809197
:105A2000E2008F7E8093E2008091E20081608093AB
:105A3000E2008091DA05882309F449C084E080936C
:105A4000DE050E9474288091E10083FF29C08091C7
:105A5000E20083FF25C08091E100877F8093E10011
:105A600082E08093DE051092DA058091E1008E7F5E
:105A70008093E1008091E2008E7F8093E20080912C
:105A8000E20080618093E20042E060E080E00E94FA
:105A90009B2B8091F00088608093F0000E946A2820
:105AA000FF91EF91BF91AF919F918F917F916F91F6
:105AB0005F914F913F912F910F900FBE0F901F90CC
:105AC000189519BC1092DE050E94672870CF80914E
:105AD000E30087FD93E09093DE05B3CF1F920F9212
:105AE0000FB60F9211242F933F934F935F936F93B1
:105AF0007F938F939F93AF93BF93CF93DF93EF9356
:105B0000FF93D091E900DF708091EC00C82FC17045
:105B100080FDC0E81092E9008091F000877F8093BB
:105B2000F00078940E94B22D1092E9008091F0006C
:105B300088608093F000CD2BCF70C093E900FF9177
:105B4000EF91DF91CF91BF91AF919F918F917F9115
:105B50006F915F914F913F912F910F900FBE0F90DA
:105B60001F9018951F93CF93DF93CDB7DEB7AA97F9
:105B70000FB6F894DEBF0FBECDBF8FED95E020913C
:105B8000F100FC012193CF01F5E0873E9F07B9F7B3
:105B90000E949C288091E80083FF1EC18091DF0550
:105BA0009091E0059A3008F017C1E92FF0E0E35436
:105BB000FF4C0C946A2F803899F0823809F00CC1A0
:105BC0008091E3058F70873008F006C18093E9006B
:105BD0008091EB0085FB882780F91092E90006C0D0
:105BE0008091DB059091DC05911182609091E80035
:105BF000977F9093E8008093F1001092F1008091DC
:105C0000E8008E77E5C0882309F4D3C0823009F01C
:105C1000E3C08091E1058111D6C08091E3058F70CA
:105C20002FEF280F263008F0D7C08093E90020918D
:105C3000EB0020FFC8C0933031F48091EB0080620C
:105C40008093EB00C0C09091EB0090619093EB00CB
:105C500021E030E001C0220F8A95EAF72093EA00A4
:105C60001092EA008091EB008860EACF8111B4C005
:105C70001091E1051F778091E3008078812B80935C
:105C8000E3008091E800877F8093E8000E94CF2B9B
:105C90008091E80080FFFCCF8091E30080688093D2
:105CA000E30082E0111183E08093DE0595C0805807
:105CB000823008F091C08091E1059091E2058C3D21
:105CC00023E09207A1F583E08A838AE289834FB7B4
:105CD000F894DE01139620E03EE051E2E32FF0E07D
:105CE00050935700E49120FF03C0E295EF703F5FAF
:105CF000EF708E2F90E0EA30C0F0C7968D939D93A1
:105D00002F5F243159F74FBF8091E800877F809340
:105D1000E8006AE270E0CE0101960E94DE2A8091DE
:105D2000E8008B778093E80057C0C096E7CF60917A
:105D3000E3057091E405AE014F5F5F4F0E94D129EA
:105D4000BC01892B09F448C09091E800977F90939B
:105D5000E80089819A810E943C2BE1CF8038E1F5EF
:105D60008091E800877F8093E8008091DA05809336
:105D7000F10045CF811130C09091E105923060F57E
:105D80008091E800877F8093E8009093DA050E9475
:105D9000CF2B8091DA05882311F084E005C0809133
:105DA000E30087FDFACF81E08093DE050E947E2824
:105DB00013C08091E105813079F481E0933009F0DE
:105DC00080E08093DC051092E9008091E800877FF5
:105DD0008093E8000E94CF2B8091E80083FF0AC0E7
:105DE0008091E800877F8093E8008091EB008062DB
:105DF0008093EB00AA960FB6F894DEBF0FBECDBF1E
:105E0000DF91CF911F9108950895CF938091DE0582
:105E10008823A1F0C091E900CF709091EC00892F08
:105E2000817090FD80E8C82B1092E9008091E80015
:105E300083FD0E94B22DCF70C093E900CF910895E9
:105E4000AA1BBB1B51E107C0AA1FBB1FA617B707A0
:105E500010F0A61BB70B881F991F5A95A9F78095BC
:105E60009095BC01CD01089597FB072E16F4009480
:105E700007D077FD09D00E94202F07FC05D03EF403
:105E8000909581959F4F0895709561957F4F0895E6
:105E9000A1E21A2EAA1BBB1BFD010DC0AA1FBB1F2E
:105EA000EE1FFF1FA217B307E407F50720F0A21BA0
:105EB000B30BE40BF50B661F771F881F991F1A940D
:105EC00069F760957095809590959B01AC01BD0137
:105ED000CF010895EE0FFF1F0590F491E02D099476
:105EE00069279627692778278727782708958F922B
:105EF0009F92AF92BF92CF92DF92EF92FF92CF9399
:105F0000DF93EC01688179818A819B81611571053C
:105F10008105910521F464E279ED8BE597E02DE1AF
:105F200033EF41E050E00E943B3049015A019B01B0
:105F3000AC01A7EAB1E40E945A306B017C01ACEEDF
:105F4000B4EFA50194010E946830DC01CB018C0DF7
:105F50009D1DAE1DBF1DB7FF03C00197A109B0482D
:105F600088839983AA83BB839F77DF91CF91FF902A
:105F7000EF90DF90CF90BF90AF909F908F9008955B
:105F80000E94772F089580E091E00E94772F089576
:105F9000B0E0A0E08093000190930101A093020182
:105FA000B09303010895FB01DC0102C005900D923E
:105FB00041505040D8F70895FB01DC0104C08D9199
:105FC0000190801921F441505040C8F7881B990B6B
:105FD0000895DC01CB01FC01F999FECF06C0F2BDAA
:105FE000E1BDF89A319600B40D9241505040B8F797
:105FF0000895F999FECF92BD81BDF89A992780B591
:106000000895A8E1B0E042E050E00C94EB2FDC01F1
:10601000A40FB51F4150504048F0CB01840F951F8D
:106020002E910E94183041505040D0F70895262FED
:10603000F999FECF92BD81BDF89A019700B402167E
:1060400039F01FBA20BD0FB6F894FA9AF99A0FBE2C
:1060500008950396272F0E9418300E941730252F8D
:106060000E941830242F0C9418300196272F0E947C
:1060700018300C941730052E97FB1EF400940E94E4
:10608000523057FD07D00E94482F07FC03D04EF432
:106090000C94523050954095309521953F4F4F4F7D
:1060A0005F4F089590958095709561957F4F8F4FC4
:1060B0009F4F08950E946D30A59F900DB49F900D45
:1060C000A49F800D911D11240895B7FF0C945A30A0
:1060D0000E945A30821B930B0895A29FB001B39F78
:1060E000C001A39F700D811D1124911DB29F700DE1
:1060F000811D1124911D0895F894FFCF92079207F6
:10610000C307C3075608F207F207F2077208D90857
:10611000E808E8084009F207F2074909BE09BE0984
:10612000C709C709C909C709C709C709BE09BE09FF
:10613000CE09C709C709CE09441A4F1A681A6D1A41
:10614000721A771A7C1A811A861A8B1A901A951A63
:106150009A1A9F1A172024204B20572062206D2066
:10616000702073207620BF20BF2079207D208520DD
:1061700092209F20A220A520B220DB2D032EEC2E02
:0E618000032EEC2E362E572EEC2EAE2EBA2EFF
:10618E000100000000FF0102030405060708090ACA
:10619E000B0C0E0F101112131415161718191A1BBB
:1061AE001C1D1E1F202122232425262728292A2BA9
:1061BE002C2D2E2F30313233343536373847393A8D
:1061CE003BFF3C3D3E3F40414243444550460D4817
:1061DE00494AFFFFFF4BFFFFFF4C4D4E4F51000052
:1061EE001E002D003C004B005A006900780087000D
:1061FE009600A500B400C300D200E000000D0F0D04
:10620E001E0D2D0D3C0D4B0D5A0D690D780D870D84
:10621E00960DA50DB40DC30DE00D001A0F1A1E1A22
:10622E002D1A3C1A4B1A5A1A691A781A871A961A84
:10623E00A51AB41AC31AE01A00270F271E272D27F6
:10624E003C274B275A276927782787279627A52784
:10625E00C327E02700341E342D343C344B345A34DB
:10626E006934783487349634A534C334D23400403C
:10627E000F401E405A409640A540B440C340D24005
:10628E00E0400404040404040404040404040404A8
:10629E0004040404040404040404040404040404B0
:1062AE0004040404040404040404040404040404A0
:1062BE000404040404040404040404040404040490
:1062CE000404040404040404040404040404040480
:1062DE0004040404C80073030300FF00FFFFB82783
:1062EE00BC272E282A282628BB270100FFFFFD7F6A
:1062FE00FF7FFF7FFF7FFF7FFF7FE200E900EA0065
:10630E00B500B600B700CD008301CC008A01920122
:10631E0094012102230224022502260227022A02C8
:10632E00B300B4006F007000818283E200E900EADE
:10633E0000B500B600B700CD008301CC008A0192F3
:10634E000194012102230224022502260227022A99
:10635E0002B300B4006F007000818283959496970B
:10636E003435366667F7F6F5F4F1F0939233323141
:10637E0030003131295A1B750A781C2E1D711D7083
:10638E001C40226DA20713073507B806D106F10689
:00000001FF
